:020000020000FC
:0200000012C02C
:02000E00AFC27F
:02001600C2C264
:100026000FED0DBF80D272D277D2DFD1EBD1DAD20B
:1000360059D278941DD000916E000023C1F0009132
:100046006600002311F000E0CDD000916700002388
:1000560011F001E0C7D000916800002311F002E022
:10006600C1D000916900002311F003E0BBD0E2CFBC
:1000760000916000003009F4089500916100013696
:1000860011F463D052C0003711F46DD04EC006375C
:1000960011F4F3D14AC0023511F4C2CF46C004367A
:1000A600B9F4009160000230F9F400916200013663
:1000B60011F486D03AC0023711F483D236C007371E
:1000C60011F4A3D232C0889485D078F1CFD02DC058
:1000D600023759F400916000023051F50091620038
:1000E60079D018F17FD021C023C0033751F4009195
:1000F60060000230E9F4009162006CD0B0F019D0D3
:1001060014C0033691F400916000033089F4009125
:10011600620060D050F010916300133411F428D0BF
:1001260004C0143411F434D000C000E00093600021
:1001360008952F931F931BE0202F1A9519F0022F75
:1001460051D0FBCF1F912F9108950FEF00936E00B2
:1001560000E000936A0000936B0000936C0000932C
:100166006D00D0D1089500E000936E00CBD10895C4
:1001760015D003D017D0C6D10895889410E00795FE
:10018600111F0795111F012F029588940795089551
:1001960005D0F3DF006206D0B5D1089595989498FE
:1001A60093980895006402BB0000969800E00DBD88
:1001B6000CBD00E808BF08B707FFFDCF969A089563
:1001C60000E054D001E052D002E050D003E04ED01F
:1001D60099D108950043043010F4889402C08ED15A
:1001E600089408951F932F93102FCAD0022D003024
:1001F60011F47CD138C009D1AAF123D19AF190BC6F
:1002060004D100E000BD00916E00002351F0012FE3
:100216009ED0202FACD0201731F100936500012F1E
:100226009CD058D1012F004D11D2012F8AD00D310B
:1002360019F0013329F014C002E408D24FD108C0E6
:100246000CE404D24BD100C0032DBFD0042DBDD089
:10025600052DBBD0062DB9D0072DB7D0082DB5D0AA
:1002660072D101C006D12F911F91089500936500A8
:1002760000E05DD0009165003DD110E3011FE6D19D
:1002860014D161D1009165007BD0192D3A2D50E033
:1002960060E006B3202F2123402F432300E00DBD4D
:1002A6000CBD00E808BF06B30123021711F05395F1
:1002B600202F06B30323041711F06395402F5436FD
:1002C60010F0643600F008B707FFEDCFF3D0052F26
:1002D600122F6FD0FBD0062F142F6BD0503031F178
:1002E600603021F10FEF202E90D002F1AAD0F2F06B
:1002F60090BC8BD000E000BD012D0D3129F4C1D09A
:10030600C4D00DE114D011C0013329F4BAD0C1D044
:1003160001E30DD00AC0003031F00F93B2D0BDD04A
:100326000F9153D0BED000E002D00DD108951F9397
:10033600CF93C6E610916500C10F0883CF911F9138
:100346000895CF93C6E6C00F0881CF910895CF9345
:10035600CAE6C00F0881CF9108951F93CF93CAE6CE
:10036600C00F109165001883CF911F91089500E08A
:100376008894030904090509060907090809089567
:100386001F932F9311E0202F003019F0111F0A95AB
:10039600FBCF912E1295A12E1124332444245524EB
:1003A600662477248824022FCCDF202E2F911F91DC
:1003B6000895003011F086D006C080D008E41030D1
:1003C60009F40CE443D1BFD008951F93102F029572
:1003D60004D0012F02D01F91089588940F70004D0C
:1003E6000A3308F0094D32D108950FEF08BB00E03B
:1003F60007BB00E000BD00E20BBF0FEF02BB0CE73E
:1004060001BB089504E00EBD08950F932F933F930B
:100416005F9330E050E0339511F4539551F020E0AE
:1004260006B30921C1F730E0532F23952B3419F079
:10043600F7CF289401C0A8945F913F912F910F9117
:1004460008952F933F934F930F9320E030E040E0C1
:1004560006B3092141F42395D9F73395C9F7439596
:10046600B9F7289401C0A8940F914F913F912F910D
:100476000895E0E4F7E064D00895EAE5F6E060D098
:100486000895EEEFF6E066D00895E8E0F7E062D072
:100496000895E2E1F7E05ED00895E0E2F7E05AD091
:1004A6000895EAE3F7E056D008950EE2CFD0CED015
:1004B600CDD00895EAEDF6E04DD00895E6EFF6E0EA
:1004C60049D00895EEEEF6E045D00895E4EEF6E064
:1004D60041D00895E8E4F7E03DD00895EEE4F7E072
:1004E60039D00895EAE6F6E02BD00895E6E5F7E080
:1004F60027D00895EEEAF6E02DD00895E0ECF6E078
:100506001FD00895E2E5F7E01BD0089500E00093C0
:10051600600000936100089500E409B906E003B99C
:1005260008E90AB9089500E00093660000936700A1
:10053600009368000093690000E000936E00089540
:1005460009D001D008950F930DE080D00AE07ED047
:100556000F9108950F93C895002021F0002D76D0B5
:100566003196F9CF0F9108950F931F931FB72F93CD
:10057600CF93C1E600916000C00F2CB1288303958C
:10058600043009F403E000936000CF912F911FBF60
:100596001F910F911895BFB6D6B2CD2CC92079F40C
:1005A60013942A9459F08894DA2009F00894881C48
:1005B600771C661C551C441C331C01C020BCBFBEE6
:1005C600189510D00091660000DF00916700FDDEEF
:1005D60000916800FADE00916900F7DE00E236D08D
:1005E60091DF0895F89410E02BD00093660011E097
:1005F60027D00093670012E023D00093680013E031
:100606001FD000936900789408950091660010E069
:100616000ED00091670011E00AD00091680012E048
:1006260006D00091690013E002D06CDF0895E199CD
:10063600FECF1EBB0DBBF894E29AE19A789408951A
:10064600E199FECF1EBBE09A0DB308955D9BFECFE8
:100656000CB9089544524F3A696E74342056302EC0
:10066600326400002A2A2A2057656C636F6D652064
:10067600746F20594144524F2D6C616E6421202ABB
:100686002A2A0D0A2863292032303036204E2E20A1
:100696004D75656C6C6572202F2F207777772E79D4
:1006A6006164726F2E646500436865636B696E678B
:1006B6002064657669636520230042616420726167
:1006C6006E67653A2072616E676520697320302E09
:1006D6002E330000436C6F636B203A2000004461A8
:1006E600746120203A2000005369676E616C000037
:1006F600737475636B2000004465766963653A2000
:10070600000037424344732027422700322A3234FE
:10071600206269747320274C2700756E6B6E6F77A5
:100726006E20747970652E2053656E64696E67203D
:100736003078000020626974730054696D656F75C6
:10074600740044524F2300003A3078004F4B0000AB
:1007560044524F2D74797065206E6F7420736574E2
:0A0766002C206E6F2044524F21003A
:00000001FF
